:020000040800F2
:10000000D00D002439030008ED170008A7170008D9
:100010004503000871050008B92000080000000031
:10002000000000000000000000000000F1170008C0
:10003000FD05000800000000EF170008A1180008E7
:100040005303000853030008530300085303000838
:100050005303000853030008530300085303000828
:100060005303000853030008530300085303000818
:100070005303000853030008530300085303000808
:1000800053030008530300085303000853030008F8
:1000900053030008530300085303000853030008E8
:1000A00053030008530300085303000853030008D8
:1000B00053030008530300085303000853030008C8
:1000C00053030008530300085303000853030008B8
:1000D0005303000875200008530300085303000869
:1000E00053030008530300080000000053030008F6
:1000F0005303000853030008530300085303000888
:100100005303000853030008530300085303000877
:100110005303000853030008530300085303000867
:100120005303000853030008530300085303000857
:100130005303000853030008530300085303000847
:1001400000000000000000000000000000000000AF
:100150005303000853030008530300085303000827
:100160005303000853030008530300085303000817
:100170005303000853030008530300085303000807
:1001800053030008530300085303000853030008F7
:1001900053030008530300085303000853030008E7
:1001A00053030008530300085303000853030008D7
:1001B00053030008530300085303000853030008C7
:1001C00053030008530300085303000853030008B7
:1001D00053030008530300085303000853030008A7
:1001E0005303000853030008530300085303000897
:1001F0005303000853030008530300085303000887
:100200005303000853030008530300085303000876
:100210005303000853030008530300085303000866
:1002200053030008530300085303000800000000B4
:1002300053030008530300080000000053030008A4
:100240005303000853030008530300085303000836
:100250005303000853030008530300085303000826
:100260005303000853030008530300085303000816
:100270005303000853030008530300080000000064
:1002800053030008000000005303000800000000B2
:10029000000000005303000800F002F800F03CF8F2
:1002A0000AA090E8000C82448344AAF10107DA45D1
:1002B00001D100F031F8AFF2090EBAE80F0013F0E7
:1002C000010F18BFFB1A43F001031847502000002C
:1002D00070200000103A24BF78C878C1FAD85207BD
:1002E00024BF30C830C144BF04680C6070470000B0
:1002F0000023002400250026103A28BF78C1FBD82F
:10030000520728BF30C148BF0B6070471FB501F0CE
:10031000EBFF1FBD10B510BD00F0E4F81146FFF76C
:10032000F5FF01F017FF00F016F903B4FFF7F2FF35
:1003300003BC01F0D2FE000009488047094800478D
:10034000FEE7FEE7FEE7FEE7FEE7FEE7FEE7FEE785
:10035000FEE7FEE704480549054A064B70470000E2
:10036000A518000899020008D0010024D00D00242F
:10037000D0030024D0030024704753EA020C00F09D
:1003800069802DE9F04B4FF00006002B1FBFB3FA38
:1003900083F503FA05F424FA05F65E4012BF16430E
:1003A000B2FA82F502FA05F4C5F120051EBF22FA61
:1003B00005FC44EA0C04203556EA044C4FEA144488
:1003C00018BF641C4FF000084FF00009904271EB19
:1003D000030C39D3002919BFB1FA81F701FA07F6E6
:1003E000B0FA80F700FA07F6C7F120071EBF20FA1F
:1003F00007FC46EA0C062037B6FBF4FCA7EB050722
:10040000103F07F01F0BCBF120060CFA0BFB2CFA68
:1004100006F644BFB3460026202FA4BF5E464FF029
:10042000000B5BEA060C08BF4FF0010B19EB0B0940
:10043000ABFB027C48EB0608C01B06FB02CC0BFBA7
:1004400003CC71EB0C01C1E70B460246414648461E
:10045000BDE8F08B13B54FF000004FF00001AFF393
:100460000080BDE81C4070470FB4044910B503AAD2
:10047000029800F009F810BC5DF814FB1400002489
:100480007047704770477047074B70B50D467B4407
:1004900000F011F80446284600F020F810B14FF0A3
:1004A000FF3070BD204670BDAF1C000001694A1CC2
:1004B00002610878704700B58FB0CDE901310021A5
:1004C000059105497944CDE903101146684600F0CD
:1004D0002EF80FB000BD0000E5FFFFFF007B00F02D
:1004E00080007047754600F03FF8AE46050069464B
:1004F000534620F00700854618B020B5FFF72AFFC5
:10050000BDE820404FF000064FF000074FF0000814
:100510004FF0000B21F00701AC46ACE8C009ACE895
:10052000C009ACE8C009ACE8C0098D4670472DE9A8
:10053000F04106460024D6E90170F5688046304651
:1005400003E04146B847641C3046A8470028F8D16C
:100550002046BDE8F08110B50446AFF30080204688
:10056000BDE81040FFF7E1BE004870476C01002471
:10057000FEE70000F0B5BFF34F8FBFF36F8F1D494B
:1005800000200860BFF34F8FBFF36F8F1A4C2168B4
:1005900041F400312160BFF34F8FBFF36F8F1649D5
:1005A00070310860BFF34F8F081F006843F6FF7576
:1005B000104E1036C0F34E31C0F3C90305EA4112A4
:1005C000184642EA80773760401EFAD2491EF5D2BB
:1005D000BFF34F8F206840F480302060BFF34F8F0F
:1005E000BFF36F8F03484C30016841F00401016094
:1005F000F0BD000050EF00E014ED00E07047000097
:1006000010B528B190F83510022903D0802141653A
:10061000012010BD1D4A4FF4956301688C189C425F
:1006200007D8042280F83520086820F0010008600F
:1006300029E00C6824F00E040C6001680A440A6882
:1006400022F001020A60016E0A6822F480720A60D8
:1006500090F85C30012202FA03F10D4B1960D0E9E9
:1006600019134B60C16E31B10B6823F480730B60BA
:10067000D0E91C134B60002180F8341080F835203D
:10068000016D01B18847002010BD0000F0FFFDBFE3
:10069000045402580248016841F0010101607047AA
:1006A000200400582DE9F84F6C4C00224FF0B04A5E
:1006B0004FF0010B4FF0030E4FF00F090B680BFAD0
:1006C00002F73B40BB4270D14D68022D01D0122D84
:1006D00012D1D50800EB850CDCF820605507ED0E33
:1006E00009FA05F826EA0806D1F8108008FA05F894
:1006F00048EA0608CCF82080D0F80080560091F82F
:1007000004C00EFA06F50CF0030C28EA05080CFAF2
:1007100006FC4CEA080CC0F800C0D1F804C0BCF1DB
:10072000010F08D0BCF1020F05D0BCF1110F02D0AF
:10073000BCF1120F16D1D0F808C0D1F80C802CEA09
:10074000050C08FA06F848EA0C08C0F80880D0F84A
:1007500004C02CEA070C0F79C7F30017974047EA4B
:100760000C074760C768AF438D68B5403D43C5601F
:100770004D68ED006BD53A4D2E6846F002062E60AE
:100780002D6822F0030606F1B04605F0020500953B
:10079000D6F808C495072F0F09FA07F52CEA050CBF
:1007A000304DA84202D100252EE050E02E4DA84247
:1007B00001D1012528E02D4DA84201D1022523E0D9
:1007C0002B4DA84201D103251EE02A4DA84201D19C
:1007D000042519E0284DA84201D1052514E0274D34
:1007E000A84201D106250FE0254DA84201D10725D9
:1007F0000AE0244DA84201D1082505E0224DA84277
:1008000001D1092500E00A25BD4045EA0C05C6F8DE
:10081000085425684E689D43F60300D51D432560A6
:1008200065684E689D43B60300D51D436560DAF8E0
:10083000005056464F689D43FF0200D51D4335606A
:1008400075684F689D43BF0200D51D437560521CFB
:10085000102AFFF433AFBDE8F88F00008000005885
:10086000F4440258000002580004025800080258DC
:10087000000C0258001002580014025800180258C8
:10088000001C0258002002580024025842694A40C5
:10089000426170470AB1018370474183704700008D
:1008A00001488068704700001800002402488168F1
:1008B000027811448160704718000024032010B5AD
:1008C00000F058F80F2000F007F808B1012010BD23
:1008D00000F022F8002010BD70B50D4D04464FF415
:1008E0007A712878B1FBF0F00A490968B1FBF0F0A1
:1008F00000F086FD48B9102C07D200222146501E78
:1009000000F018F800206C6070BD012070BD000080
:1009100018000024040000247047002809DB01218E
:1009200000F01F0291404009800000F1E020C0F873
:10093000001170470E4BF0B41B68C3F30223C3F1E0
:100940000704042C00D904241D1D072D01D2002307
:1009500000E0DB1E012606FA04F56D1E0D409D40E9
:100960009E40761E164045EA0601F0BC01F0A5BB8C
:100970000CED00E0064A00F0070110684FF6FF0397
:10098000184040EA01200349084310607047000006
:100990000CED00E00000FA0510B500F05BFA084924
:1009A00009684FF4807292FAA2F201F47061B2FA0F
:1009B00082F2D140034A515CC8400349086010BD2F
:1009C00018440258F22200080400002410B500F078
:1009D000FBF907490968102292FAA2F201F07001AE
:1009E000B2FA82F2D140034A515CC84010BD000007
:1009F00020440258F2220008364930B50A680968D6
:100A000012F00302344BC1F305311B68334C03F081
:100A100010032468DFED320AB7EE001AC4F3CC04E9
:100A200014FB03F300EE103A2E4BB8EE400A07D049
:100A30002D4C012A01D0022A4AD0B4FBF1F10BE07F
:100A4000244C283C22689506284A03D52468C4F320
:100A5000C104E240B2FBF1F101EE901A1968B8EE60
:100A6000612AC1F3080101EE901A1968F8EE611AC3
:100A700040EE201A31EE810A22EE000AC1F346212F
:100A8000491C00EE901AF8EE600A80EE201AFCEE87
:100A9000C10AC0ED000A1968C1F30641491C00EE05
:100AA000901AF8EE600A80EE201AFCEEC10AC0ED42
:100AB000010A1968C1F30661491C00EE901AF8EEAC
:100AC000600A80EE201ABCEEC10A80ED020A30BD39
:100AD000074ABFE7284402582C4402583C440258B5
:100AE000000000393844025800093D000090D0034E
:100AF00040787D01364930B50A68096812F0030272
:100B0000344BC1F305511B68334C03F480732468E4
:100B1000DFED320AB7EE001AC4F3CC0414FB03F382
:100B200000EE103A2E4BB8EE400A07D02D4C012AA9
:100B300001D0022A4AD0B4FBF1F10BE0244C283C4E
:100B400022689506284A03D52468C4F3C104E2400C
:100B5000B2FBF1F101EE901A1968B8EE612AC1F307
:100B6000080101EE901A1968F8EE611A40EE201A99
:100B700031EE810A22EE000AC1F34621491C00EE43
:100B8000901AF8EE600A80EE201AFCEEC10AC0ED61
:100B9000000A1968C1F30641491C00EE901AF8EEEC
:100BA000600A80EE201AFCEEC10AC0ED010A196845
:100BB000C1F30661491C00EE901AF8EE600A80EE5F
:100BC000201ABCEEC10A80ED020A30BD074ABFE719
:100BD000284402582C44025844440258000000396A
:100BE0004044025800093D000090D00340787D0148
:100BF0002DE9F047DFF8BC9104460E46D9F8000015
:100C000000F00700B0420CD2D9F8001021F0070123
:100C10003143C9F80010D9F8000000F00700B042D5
:100C20007ED12078DFF89081800707D5D8F80010B2
:100C3000E26821F00F011143C8F800102078C007C6
:100C400062D0D8F80010A26821F470611143C8F88E
:100C5000001059496068183902281CD003281DD09B
:100C6000096801281DD04907002960DA524F083F62
:100C7000396821F0070101433960FFF711FE05468D
:100C8000606841F28831022813D003281ED0012861
:100C90008A4627D034E009688903E5E709688901B5
:100CA000E2E7C905E0E7FFF7FBFD411B514501D92C
:100CB00023E08A463868C0F3C2000228F3D123E05B
:100CC000FFF7EEFD411B514501D916E08A46386811
:100CD000C0F3C2000328F3D116E0FFF7E1FD411B8A
:100CE00051450AD83868C0F3C2000128F5D10BE09D
:100CF000FFF7D6FD411B514502D90320BDE8F0871F
:100D0000386810F0380FF3D1D9F80010484601F0D8
:100D10000701B1420DD9016821F00701314300E01C
:100D200005E00160006800F00700B04201D001203A
:100D3000E4E72078400707D5D8F80010226921F0B1
:100D400070011143C8F80010207801071B4805D531
:100D50000168626921F07001114301602178C906C0
:100D600005D50168A26921F4E06111430160207892
:100D7000800607D51149091D0868E26920F0700056
:100D80001043086000F066F8D8F800104FF4807245
:100D900092FAA2F201F47061B2FA82F2D140084AEA
:100DA000515CC840074908600F20FFF795FD0020FF
:100DB000A4E7000000200052184402581C440258C6
:100DC000F22200080400002410B5FFF7E5FD0849F1
:100DD0000968012292FAA2F201F00F01B2FA82F23E
:100DE000D140044A515CC8400349086010BD00006E
:100DF00018440258F22200080800002410B5FFF73A
:100E0000E3FF07490968102292FAA2F201F070018B
:100E1000B2FA82F2D140034A515CC84010BD0000D2
:100E20001C440258F222000810B5FFF7CDFF074915
:100E300009684FF4807292FAA2F201F4E061B2FA0A
:100E400082F2D140024A515CC84010BD1C44025895
:100E5000F22200083548F0B50068364D10F0380130
:100E6000334809D00411082904D0334E10290BD07F
:100E700018290BD02046F0BD29688906FBD52968C2
:100E8000C1F3C101C840F0BD3046F0BD274918315B
:100E90000A68096812F00302284BC1F305111B68A8
:100EA000274F03F001033F68DFED260AB7EE001A73
:100EB000C7F3CC0717FB03F300EE103A224BB8EE52
:100EC000400A06D0012A01D0022A2BD0B4FBF1F04F
:100ED00008E02A68920603D52A68C2F3C102D0400E
:100EE000B0FBF1F001EE900A1868B8EE612AC0F389
:100EF000080001EE900A1868F8EE611A40EE201A18
:100F000031EE810A22EE000AC0F34620401C00EEBA
:100F1000900AF8EE600A80EE201ABCEEC10A10EECC
:100F2000100AF0BDB6FBF1F0DCE7000010440258F7
:100F30000090D0030044025840787D012C440258B0
:100F40003444025800000039304402582DE9F05F63
:100F500004460078DFF8FC8341F28839DFF8F8A313
:100F6000FE4DC0074ED0D8F800104046C1F3C20174
:100F700002291AD00068C0F3C200032805D1DAF8AC
:100F8000000000F0030002280FD06068B0F5803F39
:100F900012D010B1B0F5A02F19D0286820F48030FD
:100FA0002860286820F4802009E02868800329D57B
:100FB0006068002874D025E0286840F480302860FC
:100FC000606890B1FFF76CFC06464F4609E0286860
:100FD00040F480202860EFE7FFF762FC801BB842F6
:100FE0007DD828688003F7D50CE0FFF759FC06464A
:100FF0004F4604E0FFF754FC801BB842F0D8286845
:101000008003F7D42078D64F80075AD5D8F800103F
:1010100040464FF47C3B11F0380F13D00068C0F30A
:10102000C200032803D1DAF8000080070AD0E06884
:10103000A8B3296821F0190101432960FFF730FCAA
:1010400006461DE02868400702D5E0680028B1D0B8
:101050002868E16820F0190008432860FFF720FCA9
:10106000064604E0FFF71CFC801B0228B8D828685D
:101070004007F7D507E0FFF713FC801B0228AFD825
:1010800028684007F7D538689BFAABF220F47C312A
:101090002069B2FA82F290400143396011E000E029
:1010A000AEE0286820F001002860FFF7F9FB064653
:1010B00004E0FFF7F5FB801B022891D82868400761
:1010C000F7D42078C00655D5D8F8001040464FF028
:1010D000F84BC1F3C201012917D0006800E0EDE030
:1010E000C0F3C200032805D1DAF8000000F00300C5
:1010F00001280AD0E069002828682CD040F0800040
:101100002860FFF7CDFB064616E02868C00502D52B
:10111000E069802874D138689BFAABF220F0F8417E
:10112000206AB2FA82F290400143396022E0FFF770
:10113000B7FB801B022899D82868C005F7D5386806
:101140009BFAABF2216AB2FA82F220F0F8409140A9
:10115000084338600EE020F080002860FFF7A0FB15
:10116000064604E0FFF79CFB801B022887D828680E
:10117000C005F7D42078000724D5774F60694C3735
:10118000002838680FD040F001003860FFF788FB76
:10119000064604E0FFF784FB801B02288DD83868E0
:1011A0008007F7D50EE020F001003860FFF778FBEC
:1011B000064604E0FFF774FB801B02287ED83868DF
:1011C0008007F7D42078800623D5A06900282868F6
:1011D0000FD040F480502860FFF762FB064604E021
:1011E000FFF75EFB801B022868D828688004F7D5CB
:1011F0000FE020F480502860FFF752FB064605E020
:10120000D6E0FFF74DFB801B022857D828688004E2
:10121000F7D42078400744D5524F386840F48070A6
:101220003860FFF73DFB064604E0FFF739FB801B03
:10123000642843D83868C005F7D5474FA0684837B9
:1012400001280AD008B1052811D0386820F0010023
:101250003860386820F0040002E0386840F001008F
:101260003860A06888B1FFF71BFB064609E03868C4
:1012700040F004003860F0E7FFF712FB811B49459E
:101280001CD838688007F7D50BE0FFF709FB064646
:1012900004E0FFF705FB811B49450FD8386880073C
:1012A000F7D4606AF0B3D8F80010C1F3C201032983
:1012B0007ED00228286820F0807000E079E0286065
:1012C00003D0FFF7EDFA044687E0FFF7E9FA064698
:1012D00004E0FFF7E5FA801B02287BD8286880012C
:1012E000F7D4DAF8001040F2F3329143E26A41EAAF
:1012F0000211A26A1143CAF8001094F834004FF4A6
:10130000FE02218E4002491EA0F5007080B2C1F39A
:1013100008010843218F491E02EA0141084394F85D
:101320003C1000E05CE0491E120202EA0161084341
:101330000949083108600B1D19684FF6F872A06C56
:10134000914392FAA2F2B2FA82F2904001431960FC
:10135000014809E010440258284402580044025849
:101360000444025800480258001D0168226C21F014
:101370000C01114301600168626C21F0020111430C
:101380000160016841F480310160016841F400317D
:101390000160016841F480210160016841F00101B0
:1013A0000160286840F080702860FFF779FA01E05A
:1013B00018E00FE0044604E0FFF772FA001B022871
:1013C00008D828688001F7D50AE0FFF769FA001B02
:1013D000022802D90320BDE8F09F28688001F4D4D8
:1013E0000020F8E70120F6E74FF0E0210428086923
:1013F00003D020F004000861704740F00400FAE7D1
:10140000401EB0F1807F10B501D3012010BD4FF018
:10141000E02460610F21601700F04FFE0020A06102
:1014200007202061002010BD7047704790F87910A8
:1014300090F87A000843704770B502680446D06996
:101440001368916810F00F0F64D0594D03F4907633
:101450000D40354376D0C50707D0DD0505D50125FC
:101460001562E26F42F00102E267820708D5CA07FF
:1014700006D0256802222A62E26F42F00402E26787
:10148000420708D5CA0706D0256804222A62E26FFF
:1014900042F00202E26702070ED503F0200201F0DB
:1014A00080552A4352EAC17206D0256808222A6272
:1014B000E26F42F00802E267E26F002A3AD080064B
:1014C00008D503F0200001F08051084302D02046E7
:1014D00000F0D4FAE06F000703D42068806840066B
:1014E0002AD5204600F0BCFA2068816849061ED53E
:1014F000816821F040018160606FC0B12D490165B4
:10150000606FFFF77DF8002814D0606F016DBDE8B3
:1015100070400847850615D503F0200501F0805678
:1015200035430FD02046BDE8704000F0A7BA2046F2
:10153000FFF77BFF70BD05E02046FFF776FF002038
:10154000E067F7E7C6024FF020050CD54E020AD53A
:10155000E803106284F8795084F87A502046BDE898
:101560007040FFF761BF06060AD503F0800601F45C
:1015700000010E4304D02046BDE8704000F00EBDCF
:1015800041060BD5590609D51168204621F04001C6
:10159000116084F8795000F005F9CBE70002C9D555
:1015A0005800C7D5106820F080401060C2E70000E6
:1015B000010000104D1A000810B5040003D094F883
:1015C000790010B107E0012010BD002084F87800F8
:1015D000204600F027F8242084F87900206801686C
:1015E00021F001010160204600F084FA0128EBD0CF
:1015F000606B10B1204600F097F92068416821F433
:10160000904141602068816821F02A018160206852
:10161000016841F0010101602046BDE8104000F082
:10162000E7B9000010B5006886B01B49884230D188
:101630001A48016841F001010160006800F00100F2
:10164000059016481030016841F0100101600068F3
:101650000121134C00F0100005904FF40070009031
:101660000220CDE90101039007206946049020463D
:10167000FFF718F84FF48061204600916946FFF7A4
:1016800011F82520FFF749F9032225201146FFF71D
:1016900051F906B010BD000000100140E0440258AE
:1016A0000000025890F87A30202B4CD1B9B1B2B179
:1016B00090F87830012B46D0012380F878304166CD
:1016C000A0F86820A0F86A20FF228168B1F5805F49
:1016D00007D07F2351B1B1F1805F0CD010E0012021
:1016E0007047016921B940F2FF1107E0016909BBA8
:1016F000A0F86C2004E00169E1B13F21A0F86C1072
:101700000021C167222280F87A2080F878100168D1
:101710008A6842F001028A6001680A6892000CD56A
:101720000A6842F480720A600068816841F0805162
:10173000816006E0A0F86C30E2E7086840F4907041
:1017400008600020704702207047000030B5006834
:10175000114988420CD1114A5088010408D411461D
:101760004FF000034404097806D50A2901D05380BC
:1017700030BD40F400400DE00D2909D0084DC0F304
:101780000D04401C80B2C72829555080EFD830BDC9
:1017900040F48040508030BD001001401000002413
:1017A000240000247047FEE70E4810B586B001689B
:1017B00041F001010160006869460B4C00F0010036
:1017C00005900220009001200190029003200390D8
:1017D0002046FEF767FF012220460221FFF75AF854
:1017E00006B010BDE0440258000002587047704730
:1017F0007047000070B5284C9CB0256825F00405A2
:101800002560254C00260C34256845F440452560AC
:10181000256805F440451B952568AD04FCD50124D9
:1018200000940CAD03962404019402240994CDE99C
:101830000A410796082485E80D00CDE91046684660
:10184000FFF784FB88B93F2013900320CDE91406ED
:1018500040200101CDE91640CDE9180150201A9031
:10186000022113A8FFF7C4F910B101201CB070BD0C
:101870000A48016841F0800101600848F4300168BD
:1018800041F002010160006800F002001B90FEF7C9
:1018900001FF0020EAE700000C480258004402580B
:1018A000FFF704B81C48016841F4700101601B494E
:1018B000086840F001000860184A002010321060EB
:1018C0000A68174B1A400A60144A18321060121D39
:1018D0001060121D1060114A28321060121D106035
:1018E000121D1060121D1060121D1060121D10607C
:1018F000121D1060121D10600A6822F480220A6016
:1019000006496031086001200649C1F80801C00697
:10191000014980390860704788ED00E000440258B2
:101920007FEDF6EA0080005190F83410C90706D028
:1019300001684A68836B22F400321A434A6090F8C7
:101940003410890706D501684A68C36B22F48032D7
:101950001A434A6090F83410490706D501684A686E
:10196000036C22F480221A434A6090F8341009076D
:1019700006D501684A68436C22F400421A434A6063
:1019800090F83410C90606D501688A68836C22F481
:1019900080521A438A6090F83410890606D501688F
:1019A0008A68C36C22F400521A438A6090F834109B
:1019B000490611D501684A68036D22F480121A4362
:1019C0004A60016DB1F5801F06D101684A68436D18
:1019D00022F4C0021A434A6090F83410090606D572
:1019E00001684A68806D22F4002202434A60704711
:1019F000F8B500250446C567FEF752FF0746206884
:101A000000686FF07E46000708D500223B464FF481
:101A100000112046009600F0FBFA60B920680068CB
:101A200040070AD500223B464FF48001204600962D
:101A300000F0EEFA08B10320F8BD202084F8790008
:101A400084F87A00002084F87850F8BD10B5806BD7
:101A50000021A0F86A10A0F86210FFF7E6FC10BDA4
:101A600001680A6822F490720A6001688A6822F0AC
:101A700001028A60202180F87A10704710B5B0F812
:101A80006C2090F87A300168222B05D0088B40F04A
:101A900008000883022010BD898C8368B3F5805F3D
:101AA00001D103696BB11140426E531C4366117042
:101AB000B0F86A10491E0904090CA0F86A1007D092
:101AC00015E0436E11401980416E891C4166EFE7B5
:101AD00001680A6822F490720A6001688A6822F03C
:101AE00001028A60202180F87A10FFF72FFE002083
:101AF00010BD00002DE9F04F044600688025FD4B25
:101B00000021D4F810C087B0A6680F46D4F81C8016
:101B100046EA0C06D4F814C0A26A4CEA080C46EA5D
:101B20000C0632430668DFF8D0C306EA0C061643FB
:101B3000066020684268E66822F440523243426000
:101B40002268A0699A4201D0266A3043A66AB6F19B
:101B5000005F04D1D4E90B6C46EA0C06304396686A
:101B6000DFF898C306EA0C06064396602068C26A4E
:101B7000666A22F00F023243C262E14E2068E14AF7
:101B8000B04210D1126802F03802182A74D005DC75
:101B9000CAB3082A7AD0102A47D179E0202A7BD00C
:101BA000282A7CD17AE0D84EB04209D1126802F0DE
:101BB0000702062A73D2DFE802F053696B6D6F717A
:101BC000D24EB04209D1126802F00702062A66D24C
:101BD000DFE802F0465C5E606264CD4EB04209D13F
:101BE000126802F00702062A59D2DFE802F0394FE4
:101BF00051535557C74EB0420BD1126802F007023D
:101C0000062A4CD200E00EE0DFE802F02A4042440F
:101C10004648C14EB04209D1126802F03802182A73
:101C200038D0BBDCB4E74FF0010538E0BB4EB04222
:101C300009D1126802F00702062A30D2DFE802F06A
:101C40001026282A2C2EB64EB0420BD1126802F074
:101C50000702062A23D2DFE802F003191B1D1F2109
:101C600000251CE098421AD1A64A121D126802F003
:101C70000702062A13D202E00CE007E00CE0DFE8DE
:101C800002F0030507090B0D022508E0042506E014
:101C9000402504E0082502E0102500E02025DFF8BB
:101CA00064B2A04E9842DFF880A2ABF1540B73D11E
:101CB000102D31D006DC022D09D0042D0AD0082DBC
:101CC0002FD111E0202D29D0402D2AD107E0FEF799
:101CD0007DFE13E06846FEF78FFE01980EE003A834
:101CE000FEF708FF049809E0DBF800105846890663
:101CF00010D50068C0F3C1012AFA01F0002811D004
:101D00006168894601EB410181420AD8B0EB093F85
:101D100007D808E05046F3E78448F1E74FF4004065
:101D2000EEE7012733E1102D4FF000084ED006DC1E
:101D3000022D0FD0042D15D0082D04D12DE0202D1B
:101D40004AD0402D13D00127794AA0F54071914225
:101D500070D9E6E7FEF73AFE626A0023414636F89C
:101D600012200DE06846FEF747FE019803E003A845
:101D7000FEF7C0FE04980023616A36F81120194668
:101D8000FEF7FBFA62680902030241EA106150089B
:101D9000181841EB080115E032E0DBF80010584656
:101DA000890609D500680023C0F3C1012AFA01F0B1
:101DB000616A36F8112015E0606A002336F81020B9
:101DC00050460FE00023FEF7D8FABDE7606A002313
:101DD00036F81020554805E0606A002336F81020D8
:101DE0004FF400400021FEF7C8FA0902020241EA5E
:101DF00010614FEA590010184A4641EB0801E1E72B
:101E0000E3694FF4004293424DD1082D23D005DC05
:101E10008DB1012D12D0042D06D112E0102D35D038
:101E2000202D3AD0402D11D0012721F00F00C1F311
:101E3000420108435AE0FEF7E1FF16E0FEF7F4FF27
:101E400013E06846FEF7D8FD01980EE003A8FEF700
:101E500051FE049809E0DBF800105846890608D5C1
:101E60000068C0F3C1012AFA01F0616A36F8111066
:101E700010E0606A36F81010BAFBF1F041006068BB
:101E800001EB5001B1FBF0F081B2CEE7606A36F8A9
:101E900010102648B0FBF1F0F0E7606A36F8100049
:101EA000B2FBF0F0EAE7082D4AD00ADC0DB3012DB1
:101EB00043D0042D7FF44DAF6846FEF79DFD019899
:101EC00009E0102D52D0202D55D0402DF2D103A87D
:101ED000FEF710FE0498616A36F81110B0FBF1F1BC
:101EE000606801EB5001B1FBF0F080B22168C8607E
:101EF0004DE01FE0000C0058F369FFCFFFF4FF1125
:101F00000010014054440258004400400048004082
:101F1000004C004000500040001401400078004098
:101F2000007C0040022300080090D00300093D001F
:101F3000FFFC0F00FEF762FFCDE7FEF775FFCAE773
:101F4000DBF80020594692060AD50968C1F3C102A0
:101F50002AFA02F1626A36F81220B1FBF2F20FE0BF
:101F6000616A36F81120BAFBF2F209E0616A36F8CC
:101F700011200949F1E7616A36F81110B2FBF1F25C
:101F8000616802EB5102B2FBF1F189B2C16007B0A6
:101F90003846BDE8F08F000000093D0090F8791048
:101FA000212901D002207047B0F8621021B1816868
:101FB000B1F5805F13D014E001680A68920004D57F
:101FC0008A6822F400028A6003E00A6822F0800234
:101FD0000A600068016841F0400101600CE001699D
:101FE00061B1C16D4A1CC265026809781185B0F8FB
:101FF0006210491EA0F8621000207047C16D02688F
:102000000988C1F308011185C16D891CC165EEE71E
:102010002DE9F0411E46174688460446069D1CE001
:10202000681C1AD025B1FEF73BFC801BA84214D9CE
:102030002068016821F4D07101602068816821F076
:1020400001018160202084F8790084F87A00002062
:1020500084F878000320BDE8F0812068C16938EA7F
:10206000010004D00020B842DAD00020F3E70120BC
:10207000F9E7000070B50D4D00240D48FFF7DCF9BD
:1020800002E0641CAC4204D80948FFF7CFF92028CD
:10209000F7D1002402E0641CAC4206D805490122B5
:1020A0000348FFF7FFFA0028F5D170BDFFFF0100DC
:1020B000EC00002410000024FEE70907090E0028A8
:1020C00004DB00F1E02080F80014704700F00F00FE
:1020D00000F1E02080F8141D7047704710B50446E9
:1020E0000420FFF781F90148046010BD0C000024B2
:1020F00070B5002405464FF47A7603E0304600F0D0
:1021000005F8641CAC42F9D370BD000070B54FF007
:10211000E02500216C69094AAB6912685043AA693D
:102120009A42FCD002D2A3EB020302E0A4EB020627
:102130003344194413468142F1D370BD0C0000248E
:102140000349CA695206FCD5C2B20A85704700002D
:1021500000100140FEF70EFAFEF7B0FB0423022246
:102160000521A020FFF746FB4FF4C870FFF7B6FF2C
:102170004FF4E13000F09CF8FFF716FB254E0025E8
:10218000254F264C3888010416D5607024A0FEF730
:102190006BF92570274B627806E0195C3185F1698F
:1021A0004906FCD5401C207020789042F5D322A02F
:1021B000FEF75AF93D80E5E760884FF47A71401CDC
:1021C00080B26080B0FBF1F201FB120048B91CA0A4
:1021D0006580FEF749F922A0FEF746F926A0FEF732
:1021E00043F96088C821B0FBF1F201FB120010B97D
:1021F00027A0FEF739F960881E21B0FBF1F201FB40
:10220000120018B929480221FEF740FB0A20FFF707
:102210006FFFB7E700100140120000240000002407
:102220000D0AC4E3B7A2CBCDB5C4CFFBCFA23A0D04
:102230000A000000240000240D0A0D0A000000001E
:102240000D0A2053544D333248373530BFAAB7A258
:10225000B0E520B4AEBFDACAB5D1E9200D0A00005E
:102260000D0A206D63756465762E74616F62616F0F
:102270002E636F6D200D0A000D0A204465764542DD
:102280006F782020B4F3D4BDB4B4D0C2200D0A00BE
:10229000C7EBCAE4C8EBCAFDBEDD2CD2D4BBD8B3B1
:1022A000B5BCFCBDE1CAF80D0A00000000000258F0
:1022B0000B490A4A10B5C1E9002000208860C860B7
:1022C000086188610C2048610846FFF775F9BDE890
:1022D0001040044901220248FFF7E4B90010014010
:1022E000EC000024100000244FF04070E1EE100AD2
:1022F0007047000000000102030401020304060706
:102300000809010002000400060008000A000C0091
:102310001000200040008000000100003C23000865
:102320000000002424000000D402000860230008FC
:1023300024000024AC0D0000F002000800000000A2
:102340000090D0030090D0030000000000000000C7
:10235000000000000100000010000000000000006C
:040000050800029954
:00000001FF
